:100000000C941E060C94B1260C94DE260C94460625
:100010000C9446060C9446060C9446060C94460630
:100020000C9446060C9446060C9416120C94460644
:100030000C9446060C9446060C9446060C94460610
:100040000C940B270C9446060C94F92A0C943C2B28
:100050000C9446060C9446060C9446060C944606F0
:100060000C9446060C9446067217D417B317B617AD
:10007000B917BC17BF17C217C517D417CE17061963
:10008000081908190619081908190819081908196A
:100090000819081908190819081908190819081958
:1000A0008C1808190819081908190819FD170819D2
:1000B0000819081908190819081908190819081938
:1000C000081908190819081908190819981898180A
:1000D000981898189818981898189818981808192F
:1000E00008190819081908190819FD1797189718F9
:1000F000971897180819A518AB18B118B718BD1894
:10010000C318C918CF18D918E318ED18F7183E18F6
:10011000001808190819081908198C18081908195D
:1001200008190819081908190819081996189618AD
:10013000961896180819A518AB18B118B718BD1855
:10014000C318C918CF18D918E318ED18F7183E18B6
:10015000001808190819081908198C183B193B19B7
:100160003B193B193B193B193B193B193B193B19EF
:100170003B193B193B19521A521A521A521A521A67
:10018000521A80198A1994199E19FC19061A151AFF
:10019000261AAD1BC21BCE1BD71BE61B0B1C141C47
:1001A0005D1C261C541F5A1F601F671F751F971F59
:1001B000B51F456E746572206D656E752E2E2E000E
:1001C000546F67676C6564206D6963726F50504D42
:1001D00000546F67676C656420696E76657274653C
:1001E000642050504D2100546F67676C6564205443
:1001F00058206D7574696E672100546F67676C6570
:10020000642074656C656D65747279210050726F3D
:10021000746F636F6C206572726F72207769746897
:100220002052580054696D656F7574207768656E4B
:1002300020636F6E6E656374696E6720746F205201
:100240005800507265737320616E79206B65792058
:10025000746F2063616E63656C00436F6E6E6563DF
:1002600074696E6720746F2052582C20706F776508
:100270007220757020746865205258202877697440
:10028000682062696E6420706C7567206966206EF4
:100290006F74207573696E6720616C776179732064
:1002A00062696E642900546F67676C656420276912
:1002B0006D6D656469617465206F75747075742700
:1002C00000546F67676C65642027736C61766520E6
:1002D0006D6F64652700546F67676C6564202761E4
:1002E0006C776179732062696E642700546F676769
:1002F0006C65642050504D206368616E6E656C20A3
:100300006C696D69740053657420525353492069B8
:100310006E6A656374696F6E206368616E6E656C8A
:100320002028303D3D64697361626C652900536526
:10033000742050504D206D696E696D756D20737914
:100340006E630053657420626561636F6E20696E31
:1003500074657276616C0053657420626561636FC9
:100360006E2064656C617900536574206265616319
:100370006F6E206672657175656E637920696E2097
:10038000487A3A20303D64697361626C652C205074
:10039000783D504D52206368616E6E656C20782CFC
:1003A0002046783D465253206368616E6E656C202E
:1003B00078005365742050574D2073746F7020641B
:1003C000656C61792028302064697361626C6564B2
:1003D0002C20312D323535203D3D20302E317320FB
:1003E0002D2035306D696E29005365742050504DB5
:1003F0002073746F702064656C61792028302064EC
:10040000697361626C65642C20312D323535203D75
:100410003D20302E3173202D2035306D696E29003E
:10042000536574206661696C736166652064656CF0
:1004300061792028302064697361626C65642C20C6
:10044000312D323535203D3D20302E3173202D2089
:1004500035306D696E29002A2A2A2A2A2A2A2A2A50
:100460002A2A2A2A2A2A2A2A2A2A2A2A2A2A2A2AEC
:100470002A2A2A2A0052582041636B6564202D20C5
:1004800072657665727420737563636573736675E0
:100490006C21002A2A2A2A2A2A2A2A2A2A2A2A2AAD
:1004A0002A2A2A2A2A2A2A2A2A2A2A2A2A2A2A2AAC
:1004B000002A2A2A2A2A2A2A2A2A2A2A2A2A2A2AC6
:1004C0002A2A2A2A2A2A2A2A2A2A2A2A2A2A00528E
:1004D000582041636B6564202D20757064617465DC
:1004E000207375636365737366756C21002A2A2A0D
:1004F0002A2A2A2A2A2A2A2A2A2A2A2A2A2A2A2A5C
:100500002A2A2A2A2A2A2A2A2A2A0056616C696457
:100510002063686F69636573206172653A205B319F
:100520005D2D5B31365D20286368616E6E656C20E1
:10053000312D31362900536574206F7574707574D0
:1005400020666F7220706F727420005B585D2061AE
:10055000626F7274206368616E67657320616E6498
:10056000206578697420525820636F6E6669670051
:100570005B535D20736176652073657474696E6783
:100580007320746F205258005B525D20726576654F
:1005900072742052582073657474696E6773207486
:1005A0006F2064656661756C747300557365206EA9
:1005B000756D62657273205B312D445D20746F2010
:1005C0006564697420706F727473205B452D515D92
:1005D00020666F722073657474696E677300202DD6
:1005E00020726563656976657220636F6E66696700
:1005F000757261746F722C20727820737720000AF4
:100600000A6F70656E4C52536E67200053657420FC
:1006100073657269616C2062617564726174653AB8
:10062000200056616C69642063686F696365733A82
:100630002031202D20342B34202F2032202D203823
:10064000202F2033202D20382B34202F2034202D14
:10065000203132202F2035202D2031322B34202FF5
:100660002036202D20313600536574204368616E9A
:100670006E656C20636F6E6669673A20005365741F
:100680002044617461726174652028302D32293AEA
:10069000200053657420486F70206368616E6E653A
:1006A0006C7320286D61782032342C207365706162
:1006B000726174656420627920636F6D6D61732966
:1006C0002076616C69642076616C75657320312DCC
:1006D0003235353A2000536574206368616E6E656B
:1006E0006C2073706163696E6720287831306B48C5
:1006F0007A293A200053657420524620706F77653E
:10070000722028302D37293A200053657420524634
:10071000206D6167696320286865782920652E67E8
:100720002E20307844454144463030443A2000532E
:1007300065742062617365206672657175656E63AC
:10074000792028696E20487A293A20005B5A5D207A
:10075000656E746572207265636569766572206383
:100760006F6E66696775726174696F6E2075746902
:100770006C79005B465D20646973706C61792061FF
:10078000637475616C206672657175656E63696509
:10079000732075736564005B525D2063616C6375E3
:1007A0006C6174652072616E646F6D206B65792079
:1007B000616E6420686F70206C697374005B495DC2
:1007C000207265696E697469616C697A6520736508
:1007D0007474696E677320746F20736B65746368DB
:1007E0002064656661756C7473005B585D2072658A
:1007F00076657274206368616E67657320616E64EC
:100800002065786974206D656E75005B535D20739B
:100810006176652073657474696E677320746F20E8
:10082000454550524F4D20616E64206578697420B3
:100830006D656E7500557365206E756D62657273BA
:10084000205B302D395D20746F20656469742070E1
:100850006172616D657465727300202D2053797328
:1008600074656D20636F6E66696775726174696F18
:100870006E000A0A6F70656E4C52536E672000510D
:1008800029204F7574707574206265666F726520DB
:100890006C696E6B20283D465329203A2000502970
:1008A00020536C617665206D6F64652028657870D3
:1008B0006572696D656E74616C293A20004F29205C
:1008C00054696D65642042494E44206174207374FC
:1008D000617274757020203A20004E292050504DCE
:1008E000206F7574707574206C696D69746564200F
:1008F000202020203A200044495341424C454400E6
:100900004D292050504D205253534920746F20637D
:1009100068616E6E656C202020203A20004C2920F2
:1009200050504D206D696E696D756D2073796E63E1
:10093000202875732920203A200044495341424C15
:100940004544004B29204661696C736166652062ED
:100950006561636F6E20696E74762E2028312D32AA
:10096000353573293A20004A29204661696C736144
:10097000666520626561636F6E2064656C617920D5
:1009800028302D323535203D3E20313073202D204A
:100990003135306D696E293A200049292046616958
:1009A0006C7361666520626561636F6E206672714B
:1009B0002E203A200048292050574D2073746F7024
:1009C0002064656C6179202020202020203A2000BE
:1009D00047292050504D2073746F702064656C61FE
:1009E00079202020202020203A200046292046611E
:1009F000696C736166652064656C617920202020D4
:100A00002020203A200050574D206368616E6E65AB
:100A10006C200066756E6374696F6E3A2000292041
:100A2000706F72742000506F776572546F776572C3
:100A300000445446205548462033322D62697420C4
:100A400031306368004F70656E4C52536E67525878
:100A5000206D696E6920342F36636800466C7974A6
:100A6000726F6E2F4F72616E6765525820554846FF
:100A70002038636800525820747970653A20004429
:100A8000697361626C656400487A00203D3D200016
:100A900043616C63756C61746564207061636B6540
:100AA0007420696E74657276616C3A200042292068
:100AB0004D6963726F202868616C66292050504D23
:100AC000202020203A00412920496E766572746505
:100AD000642050504D20696E20202020203A0030A4
:100AE00029204D7574652062757A7A657220286DAB
:100AF0006F73746C79293A003929205365726961E2
:100B00006C2062617564726174653A00736D617224
:100B100074506F7274004672536B79005472616E38
:100B200073706172656E740044697361626C6564B0
:100B30000038292054656C656D657472793A2020FF
:100B40002020202020003729204368616E6E656CCC
:100B500020636F6E6669673A202000362920446161
:100B60007461726174652028302D32293A2020206A
:100B700000352920486F70206368616E6E656C7364
:100B80003A2020202020003429204368616E6E65C1
:100B90006C2073706163696E673A202000332920EE
:100BA000524620706F7765722028302D37293A2001
:100BB0002020003229205246206D616769633A2067
:100BC0002020202020202020003129204261736530
:100BD000206672657175656E63793A202020000089
:100BE00000000700020100000304060000000000EE
:100BF00000000001020408102040800102040810D7
:100C00002001020408102004040404040404040263
:100C10000202020202030303030303000000002395
:100C2000002600290000000000250028002B0000FD
:100C3000000000240027002A00002A2C11241FBED7
:100C4000CFEFD8E0DEBFCDBF13E0A0E0B1E0E2E639
:100C5000FEE502C005900D92AA39B107D9F716E05A
:100C6000AAE9B3E001C01D92AF35B107E1F71CE07E
:100C7000CCE3DCE004C02297FE010E94332DCA338E
:100C8000D107C9F70E94662C0C942F2F0C940000FA
:100C90008091A505813019F482E08093A5058091AB
:100CA000A505833019F484E08093A5050895A895DF
:100CB0000895DC01ED91FC910190F081E02D099502
:100CC000089561E083E10E940E2860E083E10E94C4
:100CD000472882E08093B00085E08093B10061E016
:100CE00083E00E940E2860E083E00E944728089578
:100CF000A4E0B0E0EEE7F6E00C940A2D009749F18D
:100D00009C0140E050E068E478EE81E090E00E94D1
:100D1000DB2C61E083E129833A834B835C830E946F
:100D200047282981822F3A81932F4B81A42F5C8100
:100D3000B52F8F3F9105A105B10529F020F08FEF68
:100D400090E0A0E0B0E08093B3008091B0008061BB
:100D500007C060E083E10E9447288091B0008F7E49
:100D60008093B0002496E2E00C94262D60E08CE0A5
:100D70000E940E2861E08BE00E940E2861E08DE069
:100D80000E940E2860E082E00E940E2861E084E06C
:100D90000E940E28089542E050E068E476E080E08A
:100DA0000E9491260895E3E0F0E089E080935700E7
:100DB000E491E67081E0E63009F080E00895CF9399
:100DC000DF93C82F0E94D306882381F0DFB781E02C
:100DD0008093A405F8940E94570688E180936000F0
:100DE000C0936000C1110E945706DFBFDF91CF9111
:100DF00008952091440530914505382748E0C90100
:100E0000880F991F37FF06C09C0151E2252750E14A
:100E1000352701C09C01415091F73093450520933F
:100E200044050895D82FC0E0CD1780F4439A64E6B6
:100E300070E080E090E00E948427439864E670E0D0
:100E400080E090E00E948427CF5FEECF6CE271E0FB
:100E500080E090E00E948427E6CF0F931F93CF930A
:100E6000DF93EC01062F15E0115051F0CE010E94E6
:100E7000162F081741F0602FCE010E941E2FF4CFCD
:100E800082E00E941207DF91CF911F910F91089588
:100E9000A0E0B0E0EEE4F7E00C94FC2C482E562ED7
:100EA000C0E0D0E0612C712CE12CF12C00E010E0CE
:100EB00041100CC06090A30586E4689E30011124A7
:100EC000A9E1EA2EF12C0AE815E01EC091E04912D2
:100ED0000FC06090A305E6E46E9E30011124FBE193
:100EE0006F0E711CF9E2EF2EF12C06E415E00CC038
:100EF00082E0481209C078E1672E77247394EE24CB
:100F0000E394F12C03EA15E043018C0E9D1E109230
:100F10004505109244053401A62CA818B12CC30134
:100F200001966C01AE14BF04A8F4A00EB11E5110BE
:100F300006C0C3010E94162FF501808305C0F5018C
:100F40006081C3010E942D07F50180810E94F9068E
:100F50003601E2CFC301511018C0C3010E94162F01
:100F6000B82EC6010E94162F2B2D30E0322F2227DB
:100F7000282B80914405909145058217930779F4B9
:100F8000C0E0D0E05524539493CF360160914505DD
:100F90000E942D0760914405C6010E942D07C05E86
:100FA000DE4FC13E92E0D90708F482CF852DCDB740
:100FB000DEB7E0E10C94182D87E38093460580E0CE
:100FC00092ECA1E0B0E08093470590934805A09390
:100FD0004905B0934A0587E08093530580EC92E978
:100FE000ADEEB9E180934B0590934C05A0934D0570
:100FF000B0934E0585E0809354058DEE9EEFADEAEB
:10100000BEED80934F0590935005A0935105B0938A
:101010005205E5E5F5E080E090E0863028F4DC015B
:10102000AC59BC4F2C9101C020E02193019688312E
:10103000910599F782E080936D058AE080936E05B3
:10104000089561E082E00E944807089560E082E030
:101050000E9448078091A305843020F01092A305D8
:101060000E9421080895A1E0B0E0E9E3F8E00C94C3
:101070000A2D89830E9426089091A30589819817DB
:1010800031F0843020F48093A3050E94210821963A
:10109000E2E00C94262D80EC91EDA8E9BBE1809371
:1010A0008B0590938C05A0938D05B0938E0580E001
:1010B00090E0A0E0B0E580938F0590939005A09319
:1010C0009105B0939205E3E9F5E080E081938F5FAD
:1010D0008031E1F70895A0E0B0E0E1E7F8E00C949A
:1010E000002D0E9461276115710581059105C9F3E5
:1010F0000E949F2D10924F0510925005109251059D
:1011000010925205C4E0C12CD12C7601CA94809073
:101110004F0590905005A0905105B0905205BA2C03
:10112000A92C982C88240E949A2DA70196010E9430
:10113000DB2C680D791D8A1D9B1D60934F057093F4
:1011400050058093510590935205C15001F705E574
:1011500015E0E801C12CD12CB2E38B2E912CA12CEF
:10116000B12C80E1E82E87E2F82E8881882309F4EB
:1011700046C0D39419F40E94DC0741C00E949A2D06
:10118000A50194010E94DB2C21E0260FE5E5F5E0A6
:101190008E2F801B8C1520F481918213F9CFE9CF1B
:1011A00040915405249FA00111244E9DC0014F9DE4
:1011B000900D5E9D900D1124AA2797FDA095BA2F42
:1011C00040914B0550914C0560914D0570914E0535
:1011D000840F951FA61FB71F40918B0550918C055A
:1011E00060918D0570918E05481759076A077B0736
:1011F00008F4BFCF2993C39488E1C812B6CFCDB706
:10120000DEB7ECE00C941C2D61E080E00E94480702
:1012100061E081E00E944807089560E080E00E945C
:101220004807882331F060E081E00E94480781117F
:1012300008C00E944B080E94DC070E946B080E94B5
:10124000040908958436910520F4BC0180E090E003
:1012500017C09C018E3B910528F42A553109AAE05C
:10126000B0E00CC0823D910528F4245B3109A4E66E
:10127000B0E004C02D5C3109A8E5B2E00E94732CF7
:10128000A4E6B0E09B01AC010E94822C089590E09E
:101290008C599F4F0E94220908958F929F92AF927E
:1012A000BF92CF92DF92EF92FF92CF93FC01C0A545
:1012B000EC2FE770F0E0E45BFC4FA081B0E0C7FFEB
:1012C00003C024E130E002C02FE030E0FC0197A130
:1012D00083E1989FF0011124E25CFE4F80809180B1
:1012E000A280B380A20FB31F20E43FE14DE750E09E
:1012F0000E948D2CA50194010E94B92C8C2F88711D
:1013000049F469017A01E0EDCE0EE7E0DE1EE11C52
:10131000F11C1BC0C7FF05C060E47AE88CE29EE0C8
:1013200004C060E07EEE8AEB9BE069017A01F8EB95
:10133000CF0EFBE0DF1EE11CF11CA50194010E9411
:10134000B92CC20ED31EE41EF51EC701B6016951A9
:101350007C4F8F4F9F4F28EE33E040E050E00E94DB
:10136000B92CA8EEB3E00E94822CCF91FF90EF90B1
:10137000DF90CF90BF90AF909F908F9008958F3F58
:10138000910551F048F0811522E0920738F081155F
:10139000934030F482E0089580E0089581E008955C
:1013A00083E00895A0E0B0E0E8EDF9E00C94052DAD
:1013B000EB018A01B82FB695A0E028813981F801A8
:1013C00020832A813B8121832C813D8122832E81B0
:1013D0003F812383688179814A815B812C813D81B2
:1013E000EE81FF819F2F9295990F990F907C272F67
:1013F0002370922B252F2370220F220F922B232F45
:1014000023702295207F922BF80194830B5F1F4F4E
:101410002896AF5FBA1788F680FF24C0888199812B
:101420000E94BF09D82E8A819B810E94BF09E82EA5
:101430008C819D810E94BF09F82E8E819F810E9420
:10144000BF09F0E4DF9EA001112490E1E99E900124
:101450001124242B282BE4E0FE9EB0011124262B1E
:10146000F8012083CDB7DEB7E7E00C94212D803260
:1014700023E0920708F1883E23E0920740F48F5161
:101480009340E4E096958795EA95E1F70895803DCD
:1014900027E0920718F48C5D93400895883928E07E
:1014A000920768F4885C974074E0969587957A95E2
:1014B000E1F78D509C4F089580E090E008958FEF04
:1014C00093E008958C30910540F4A4E0880F991FB3
:1014D000AA95E1F7885D9C4F0895843F23E0920729
:1014E00018F484529C4F0895811524E0920740F42B
:1014F0008657934FF4E0880F991FFA95E1F7089506
:1015000080E998E008959C013695279525753575F5
:10151000821B930B9C012373337396958795969545
:10152000879583739373820F931F9C0154E03695C4
:1015300027955A95E1F7280F391F2F703F7041E02A
:1015400051E0249FC001259F900D349F900D1124E0
:10155000892F08952D98882319F000002B9A02C036
:1015600000002B9800002D9A000008952D9A00008D
:1015700083B12D980000829581700895CF93DF93F9
:10158000D82F5C9A2D985C98C8E08D2F80780E94A7
:10159000AA0ADD0FC150C9F72D98DF91CF910895A8
:1015A0008F770E94BE0A0895CF93DF93D82FC8E0AB
:1015B0008D2F80780E94AA0ADD0FC150C9F72D989F
:1015C000DF91CF910895CF93DF932D98C8E080E00D
:1015D000D82FDD0F0E94B60A8D0FC150C9F7DF91D9
:1015E000CF9108950E94D00A0E94E30A5C9A089560
:1015F000A1E0B0E0EEEFFAE00C940A2D8068698378
:101600000E94BE0A6981862F0E94D40A5C9A2196A4
:10161000E2E00C94262DCF93C0914F05C827E82F08
:10162000F0E0EA5BFA4F678589E70E94F80A6C2FC1
:101630008DE30E94F80A6C2F82E40E94F80ACF9191
:10164000089586E20E94F20A0895CF93DF93EC0199
:101650006C818CE10E94F80A6D818DE10E94F80A8C
:101660006E818EE10E94F80A6F8180E20E94F80A82
:10167000688581E20E94F80A698582E20E94F80A80
:101680006A8583E20E94F80A6B8584E20E94F80A68
:101690006C8585E20E94F80A6D858AE20E94F80A4C
:1016A0006E858EE60E94F80A6F858FE60E94F80A22
:1016B000688980E70E94F80A698981E70E94F80A30
:1016C0006A8982E70E94F80ADF91CF910895CF924C
:1016D000DF92EF92FF92CF93DF936B017C01C114F5
:1016E00088E3D8068CE9E8068CE1F80628F5C701FE
:1016F000B60120E836E948E950E00E94B92CE9013A
:10170000689760E879E687E69FEF0E94952C6C0D5C
:101710007D1D8E1D9F1DF2E0660F771F881F991F8C
:10172000FA95D1F721E732E040E050E00E94B92C71
:10173000F22EE32E80E421C0C701B60120E03DE295
:1017400041E351E00E94B92CE901689760E073ED34
:101750008EEC9EEF0E94952C6C0D7D1D8E1D9F1DA5
:10176000660F771F881F991F21E732E040E050E0A5
:101770000E94B92CF22EE32E80E66C2F6F71680F59
:1017800085E70E94F80A6E2D86E70E94F80A6F2D01
:1017900087E70E94F80ADF91CF91FF90EF90DF90EA
:1017A000CF900895682F8DE60E94F80A08958F92D1
:1017B0009F92AF92BF92CF92DF92EF92FF92CF9320
:1017C000DF93D82F83E00E94F20A8093430584E0E0
:1017D0000E94F20A8093420560E086E00E94F80AC7
:1017E00061E087E00E94F80A6FE789E00E94F80A4A
:1017F00065E08AE00E94F80A62E18BE00E94F80A44
:1018000065E18CE00E94F80A6DEF8DE00E94F80A15
:1018100060E08EE00E94F80ADD2319F08BE291E08F
:1018200008C020916D0533E1239FC0011124825C23
:101830009E4F0E94250B6CE880E30E94F80A6FE03F
:1018400082E30E94F80A62E483E30E94F80A80912E
:101850006E0587FF02C064E101C06AE084E30E9474
:10186000F80A6AE285E30E94F80A6DE286E30E94C4
:10187000F80A64ED87E30E94F80A60E088E30E94BA
:10188000F80A60E089E30E94F80AD11109C0C0900B
:101890004F05D0905005E0905105F090520507C0DB
:1018A000C5E8CC2EC1ECDC2EED2CCEEDFC2ECAE32F
:1018B0008F2C9924AA24BB24682D8C2F0E94F80A0F
:1018C000682D85E08C0F0E94F80AFE2CED2CDC2C94
:1018D000CC24CF5FCE3361F76FEF83E40E94F80A28
:1018E0006FEF84E40E94F80A6FEF85E40E94F80A23
:1018F0006FEF86E40E94F80ADD2311F066E002C073
:10190000609153058DE60E94F80A60E089E70E9425
:10191000F80A609154058AE70E94F80A60E083E7BC
:101920000E94F80A60E084E70E94F80AD11109C019
:1019300060914B0570914C0580914D0590914E053D
:1019400004C060EC72E98DEE99E10E94670BDF91B3
:10195000CF91FF90EF90DF90CF90BF90AF909F908E
:101960008F90089561E087E00E94F80A64E28EE7B4
:101970000E94F80A63E088E00E94F80A60E088E0CC
:101980000E94F80A65E087E00E94F80A62E085E0BC
:101990000E94F80A83E00E94F20A8093430584E0E3
:1019A0000E94F20A80934205089583E00E94F20AA1
:1019B0008093430584E00E94F20A8093420561E02F
:1019C00087E00E94F80A6AE070E080E090E00E9400
:1019D00084270E94B20C00000895CF92DF92FF92FC
:1019E0000F931F93CF93DF931F92CDB7DEB7082FCE
:1019F000162F8EE399830E94F80AF02EC02E99814B
:101A0000D92E8C2D8F19811738F4F60161916F0151
:101A10008FE70E94F80AF5CF64E085E00E94F80A9B
:101A200083E00E94F20A8093430584E00E94F20A58
:101A3000809342050E94612760933E0570933F05A5
:101A4000809340059093410569E087E00E94F80A81
:101A500081E08093A5050F90DF91CF911F910F91A9
:101A6000FF90DF90CF9008950F931F930E94ED0C8D
:101A70008091A505813099F40E94612700913E056F
:101A800010913F052091400530914105601B710B7D
:101A9000820B930B603A76488140910548F3809120
:101AA000A505813031F46EE971E083EB95E00E9489
:101AB0004D291F910F9108950F931F938091A505B4
:101AC000823021F41092A50581E020C08091A50507
:101AD0008130D9F40E94612700913E0510913F05A5
:101AE0002091400530914105601B710B820B930BD7
:101AF000613A76488140910540F061E087E00E94BC
:101B0000F80A1092A50582E001C080E01F910F91B4
:101B10000895CF93DF93EC014AE050E06D2F70E021
:101B200083EB95E00E941B2A6EE283EB95E00E9416
:101B30001F29BE0184E0769567958A95E1F76F705D
:101B400077274AE050E083EB95E00E941B2A6EE283
:101B500083EB95E00E941F29BE016F7077274AE052
:101B600050E083EB95E00E941B2ADF91CF9108950E
:101B7000882319F06AEA71E002C06EEA71E083EB33
:101B800095E00E944D290895FF920F931F93CF93E4
:101B9000DF9369EC7BE083EB95E00E94F9284091AC
:101BA0004B0550914C0560914D0570914E052AE012
:101BB00030E083EB95E00E94222A63EB7BE083EB2D
:101BC00095E00E94F92840914F0550915005609191
:101BD00051057091520520E130E083EB95E00E94C1
:101BE000222A6DE97BE083EB95E00E94F9284AE028
:101BF00050E06091530583EB95E00E944A2A67E824
:101C00007BE083EB95E00E94F9284AE050E0609188
:101C1000540583EB95E00E944A2A61E77BE083EB61
:101C200095E00E94F928C5E5D5E0F12C8E01888168
:101C30008823A9F0FF2031F061EB71E083EB95E0A0
:101C40000E941C2921964AE050E0F801608183EB54
:101C500095E00E94132AF394F8E1FF12E7CF83EB9B
:101C600095E00E9427296BE57BE083EB95E00E94DD
:101C7000F9284AE050E060916D0583EB95E00E9401
:101C80004A2A66E47BE083EB95E00E94F928E09124
:101C90006E05E770F0E0EE0FFF1FEC5AFC4F60811D
:101CA000718183EB95E00E944D2961E37BE083EB3A
:101CB00095E00E94F92880916E058871883069F05E
:101CC00028F4811113C068E27BE00CC0803141F040
:101CD000883161F46CE07BE005C06CE17BE002C020
:101CE00066E17BE083EB95E00E943B2968EF7AE0B8
:101CF00083EB95E00E94F9284091470550914805F3
:101D00006091490570914A052AE030E083EB95E047
:101D10000E94222A6FED7AE083EB95E00E94F92879
:101D200080918F0580710E94B80D66EC7AE083EB9C
:101D300095E00E94F92880918F0580740E94B80D6B
:101D40006DEA7AE083EB95E00E94F92880918F0597
:101D500080720E94B80D60E97AE083EB95E00E9402
:101D6000F92886E495E00E944D09AB01BC012AE008
:101D700030E083EB95E00E94042A6BE87AE083EB85
:101D800095E00E94F92886E495E00E944D099B01A8
:101D9000AC0160E472E48FE090E00E94B92CBA01DB
:101DA000A9012AE030E083EB95E00E94042A68E86C
:101DB0007AE083EB95E00E943B29CDB7DEB7E5E002
:101DC0000C94232D8F929F92AF92BF92CF92DF926D
:101DD000EF92FF92811107C06FE77AE083EB95E005
:101DE0000E943B292FC090E00E94220924E630E0A7
:101DF00040E050E00E94B92CCA01B9012AE030E06D
:101E000040E050E00E94B92C49015A016B017C016D
:101E10002AE030E0B501A40183EB95E00E94042A9A
:101E20006EE283EB95E00E941F292AE030E0B701C3
:101E3000A60183EB95E00E94042A63E783EB95E01B
:101E40000E945F29FF90EF90DF90CF90BF90AF90FE
:101E50009F908F9008951F93CF93DF9365E77AE06B
:101E600083EB95E00E94F92880916F05813041F461
:101E70006CE57AE083EB95E00E943B2910E050C0CE
:101E8000823019F465E47AE0F5CF843019F461E327
:101E90007AE0F0CF853091F766E27AE0EBCFC12FA0
:101EA000D0E0C930D1050CF441C068E3610F83EB89
:101EB00095E00E941F296EE17AE083EB95E00E9495
:101EC000F928BE016F5F7F4F4AE050E083EB95E059
:101ED0000E94E32963E17AE083EB95E00E94F92810
:101EE000C159DA4FE981E03218F566E07AE083EB18
:101EF00095E00E94F9288981803130F06FE373E02A
:101F000083EB95E00E941C2969816F7070E06F5F20
:101F10007F4F4AE050E083EB95E00E94EC291F5F81
:101F200080911A05181708F4BACF0FC061E3BECF2D
:101F3000EF70F0E0EE0FFF1FE659FC4F60817181FA
:101F400083EB95E00E944D29EACF6BEE79E083EBBD
:101F500095E00E94F928809187050E94E20E60EDCD
:101F600079E083EB95E00E94F928809188050E9432
:101F7000E20E65EB79E083EB95E00E94F928809111
:101F800089050E94E20E6AE979E083EB95E00E9400
:101F9000F92840917F0550918005609181057091ED
:101FA0008205411551056105710539F12AE030E0DE
:101FB00083EB95E00E94222A67E679E083EB95E0C7
:101FC0000E94F928809183050E944709AB01BC015A
:101FD0002AE030E083EB95E00E94222A63E479E076
:101FE00083EB95E00E94F9284AE050E06091840577
:101FF00083EB95E00E944A2A06C06AE379E083EB0E
:1020000095E00E943B296DE179E083EB95E00E9429
:10201000F92860918505709186054AE050E083EBD0
:1020200095E00E94342A60E079E083EB95E00E941D
:10203000F92860917E05603450F470E06F5F7F4F47
:102040004AE050E083EB95E00E94EC2906C067EF80
:1020500078E083EB95E00E943B296AED78E083EB22
:1020600095E00E94F92880917D0580FF03C063EB15
:1020700071E002C067EB71E083EB95E00E944D29AF
:102080006DEB78E083EB95E00E94F92880917D0567
:1020900082700E94B80D6EE978E083EB95E00E94B3
:1020A000F92880917D0584700E94B80D6FE778E073
:1020B00083EB95E00E94F92880917D0588700E944D
:1020C000B80DDF91CF911F9108950F931F93CF9378
:1020D000DF93209117052F3FA9F56FEF75E083EB94
:1020E00095E00E94F92884E793E00E94890D6EED47
:1020F00075E083EB95E00E94F92880911805909196
:1021000019050E94890D6BEA75E083EB95E00E944A
:102110003B2968E875E083EB95E00E943B2960E786
:1021200075E083EB95E00E943B296BE475E083EB5F
:1021300095E00E943B2983EB95E00E9427290E94AD
:102140002B0F68C012160CF065C0332727FD3095A1
:1021500080911A0590E0821793070CF45BC066E348
:1021600075E083EB95E00E94F928609117057727C9
:1021700067FD70954AE050E083EB95E00E94EC2902
:102180006BE075E083EB95E00E94F92810E008E22F
:1021900080911B051817D0F5C12FD0E0CC0FDD1FA3
:1021A000C45EDA4F288130E080911705992787FDBA
:1021B000909501972817390739F56BEB71E083EBA0
:1021C00095E00E941C294AE050E0602F83EB95E0E7
:1021D0000E94132A6FEB71E083EB95E00E941C29AB
:1021E000E981EF70F0E0EE0FFF1FE659FC4F6081D0
:1021F000718183EB95E00E941C2963EC71E083EB15
:1022000095E00E941C290F5F1F5FC2CF83EB95E012
:102210000E942729DF91CF911F910F910895FF927E
:102220000F931F93CF93DF93C5E5D5E0F12C8E017B
:1022300088818823D1F165EC71E083EB95E00E9401
:102240001C294AE050E06F2D83EB95E00E94132A91
:1022500062ED71E083EB95E00E941C292196F80164
:10226000208130E0A0E1B7E20E94732C9B01AC0119
:10227000A0915405B0E00E94822CAB01BC0180917A
:102280004B0590914C05A0914D05B0914E05480F1E
:10229000591F6A1F7B1F2AE030E083EB95E00E9404
:1022A000222AF394F8E1FF12C2CFCDB7DEB7E5E002
:1022B0000C94232D1092B10485E6E2EBF4E0DF01EB
:1022C0001D928A95E9F70895CF93C82F8F3719F09B
:1022D000883009F045C0E091B104EE23D9F1E15016
:1022E000E093B104F0E0EE54FB4F10826DE070E03B
:1022F00083EB95E00E945906C0E08091B104C817B5
:1023000060F4EC2FF0E0EE54FB4F608170E083EB63
:1023100095E00E945906CF5FF0CF60E270E083EB5A
:1023200095E00E9459066DE070E083EB95E00E9415
:102330005906C0E08091B104C81778F5EC2FF0E0A1
:10234000EE54FB4F608170E083EB95E00E945906EC
:10235000CF5FF0CF67E083EB95E00E941F291DC09F
:102360008B3119F40E945A111AC08D30C1F08A3095
:10237000B1F08091B104843668F76C2F70E083EB84
:1023800095E00E945906E091B10481E08E0F8093A0
:10239000B104F0E0EE54FB4FC08380E001C081E067
:1023A000CF910895CF93C82F0E94612760939A041C
:1023B00070939B0480939C0490939D04C093AF04FE
:1023C000CC2329F040E051EE60E070E004C040E82A
:1023D00055E260E070E083EB95E00E94A92BCF917D
:1023E000089590919E04492F4F7050E0BA016F5F9D
:1023F0007F4F292F30E0E4E035952795EA95E1F706
:102400006217730759F0FA01E156FB4F808381E0B0
:10241000890F8F70907F892B80939E0408956EE7BB
:1024200070E083EB95E00E94590608951F920F9289
:102430000FB60F9211241F932F933F934F935F93E7
:102440006F937F938F939F93AF93BF93CF93DF93BC
:10245000EF93FF93C0918600D0918700809159043B
:1024600090915A0420917B04211155C09E01281B94
:10247000390B80918F0590919005A0919105B091B5
:10248000920585FD02C036952795253C49E0340725
:10249000B8F140910A0150E060E070E01CE1B695AF
:1024A000A795979587951A95D1F70097A105B1053E
:1024B00021F481E090E0A0E0B0E084179507A60742
:1024C000B707D8F480910A018F3FB9F040E08091BE
:1024D0000A01481780F4842F90E0880F991FFC01AF
:1024E000E55AFB4F20813181FC01E55FFE4F3183CE
:1024F00020834F5FECCF10927C0410920A010BC036
:102500002D3B82E0380720F080910A018031D8F01D
:102510008FEF80930A01D0935A04C0935904FF911E
:10252000EF91DF91CF91BF91AF919F918F917F916B
:102530006F915F914F913F912F911F910F900FBE1F
:102540000F901F90189510910A0181E0810F8093E0
:102550000A01C9010E94370AE12FF0E0EE0FFF1FC8
:10256000E55AFB4F91838083D6CF83E08093800030
:102570008AE98093810080918F0586FD05C0809156
:1025800081008064809381008FEF9FEF909389009A
:102590008093880080916F00806280936F0008951F
:1025A0006F3018F086958058089589E0689F802DD7
:1025B00011240895A0E0B0E0E0EEF2E10C94042DC7
:1025C000C82F0E94612700910A0410910B042091EA
:1025D0000C0430910D046B017C01C01AD10AE20A8F
:1025E000F30A9701860149E8C41643E1D406E104E1
:1025F000F10410F010920E0460930A0470930B041F
:1026000080930C0490930D0420917B048FEF820F34
:102610008230D8F5E0910E04EE2309F44EC1E1308A
:1026200011F482E0B8C1E03108F034C181E08E0FCE
:1026300080930E04F0E0E55AFB4FC083803109F02F
:10264000ACC1EDE5F4E0213029F4A181A695A69571
:10265000808108C080819181A92FA695A695A69515
:1026600096958795A03148F4B0E090E0AA0FBB1F83
:10267000A55FBE4F11969C938E9310927C04329668
:1026800084E0EB36F807F9F688C1233009F005C17C
:10269000E0910E04E11104C0CF3009F07EC10DC1FC
:1026A000E83148F481E08E0F80930E04F0E0E65AA2
:1026B000FB4FC08372C1E83109F0ECC0C111EAC020
:1026C00040E050E0ABE0CA01B3E0880F991FBA9533
:1026D000E1F7A49F9001A59F300D1124F901E55A5F
:1026E000FB4F6081E1817E2F777075956795FC01C6
:1026F000EE0FFF1FE55FFE4F71836083F901E45A1F
:10270000FB4FB081B695B695B695E181FE2FF29557
:10271000FF0FF07E6F2F6B2BE695E695E6957E2FEB
:10272000777075956795FC01EE0FFF1FE35FFE4F15
:1027300071836083F901E35AFB4FB081B295B6957E
:10274000B695B370C181DC2FDD0FDD0F6D2F6B2BC4
:10275000C295C695C695C370E281E170EE0FEE0F8B
:102760007E2F7C2B75956795FC01EE0FFF1FE15FB7
:10277000FE4F71836083F901E15AFB4FB081B6953A
:10278000E181FE2FF795FF27F7956F2F6B2BE695CD
:102790007E2F777075956795FC01EE0FFF1FEF5E3A
:1027A000FE4F71836083F901E05AFB4FB081B2950F
:1027B000BF70E181FE2FF295F07F6F2F6B2BE295BA
:1027C000EF707E2F777075956795FC01EE0FFF1FF8
:1027D000ED5EFE4F71836083F901EF59FB4FB081CD
:1027E000BB1FBB27BB1FC181DC2FDD0F6D2F6B2BE8
:1027F000CC1FCC27CC1FE281E370EE0F7E2F7C2B09
:1028000075956795FC01EE0FFF1FEB5EFE4F718320
:102810006083F901ED59FB4FB081B695B695E18122
:10282000FE2FF295FF0FFF0FF07C6F2F6B2BE695BD
:10283000E6957E2F777075956795FC01EE0FFF1F6B
:10284000E95EFE4F71836083F901EC59FB4F2081F3
:102850002295269527703181E32FEE0FEE0FEE0FB4
:102860006E2F622B732F729576957770759567959D
:10287000FC01EE0FFF1FE75EFE4F718360834F5F29
:102880005F4F4230510509F01ECF8091710483FFE4
:1028900010927C0410920E0480C0243009F07DC098
:1028A00060910E0461110BC0C83AB1F41092450555
:1028B0001092440588EA0E94F90681E06CC06130FC
:1028C00019F4C093090404C0623031F4C0930804C1
:1028D0008C2F0E94F9065AC0E09108042E2F30E098
:1028E000220F331F462F50E0C90102968417950727
:1028F0003CF0633268F7FA01E85AFB4FC083E8CF37
:102900002D5F3F4F8C2F90E06091440570914505FD
:102910004217530749F4982F8827862797279093C3
:1029200045058093440532C06817790769F58091A1
:102930000904813049F5E13118F080E18093080401
:10294000F0900804CCE5D4E000E010E00F15D0F4DE
:10295000FE013197808190E0982F88272881822B73
:1029600063E0969587956A95E1F70E94370AF8012A
:10297000EE0FFF1FE55FFE4F918380830F5F1F4FB8
:102980002296E4CF10927C0410920E0480910E04E3
:10299000882319F08F5F80930E04CDB7DEB7E8E08F
:1029A0000C94202DE82FF0E0E657FA4FE185E03156
:1029B00058F4F894F0E0EE0FFF1FE55FFE4F208122
:1029C00031817894C9010895E03121F0E13131F489
:1029D00083E101C082E10E94A328089580E092E093
:1029E0000895A2E2B0E0E7EFF4E10C94FA2C9E0126
:1029F0002F5F3F4F80E1D9011D928A95E9F766ED7F
:102A000071E083EB95E029A33AA30E944D290E942F
:102A1000D50C1D8A1E8A1F8A188E312C212C00E0AD
:102A2000812C912C540170E4472E71EE572E7DE9D4
:102A3000672E78E1772EE0E5CE2EE3ECDE2EE12C5A
:102A4000F12C84EF91E0A0E0B0E08D8F9E8FAF8FEE
:102A5000B8A380EC91EDA8E9BBE1898F9A8FAB8F89
:102A6000BC8F80E491EEADE9B8E1898B9A8BAB8B9A
:102A7000BC8B83EB95E00E94612A892B09F4E1C0AD
:102A800083EB95E00E948E2A9C0133272C3231057E
:102A900009F442C0ACF42332310509F0ABC019820D
:102AA0001A821B821C821D821E821F821886198632
:102AB0001A861B861C861D861E861F86188A60C085
:102AC0002434310529F02335310509F4B2C092C010
:102AD00064E483EB95E00E941F292AE030E040E4A3
:102AE00051EE6DE978E183EB95E00E94AD296CE24F
:102AF00083EB95E00E941F292AE030E040EC51ED85
:102B000068E97BE183EB95E00E94AD296CE283EB01
:102B100095E00E945F29ADCF0F5F043009F0A9CF87
:102B200029813A814B815C81A8EEB3E00E94822C1E
:102B3000698B7A8B8B8B9C8B2D813E814F81588545
:102B40000E94822C698F7A8F8B8F9C8F29853A8582
:102B50004B855C852D8F3E8F4F8F58A32D853E85ED
:102B60004F8558890E94822C6B017C0160323EE4C3
:102B700073078105910530F462E38CE10E94F80A45
:102B800000E077CF603345E774078105910510F4C5
:102B900062E2F3CF60345CE975078105910510F4BA
:102BA00066E2EBCF80E5C81683ECD806E104F104B9
:102BB00010F462E1E2CF90E6C9169AEED906E1047C
:102BC000F10410F465E1D9CFA0E7CA16A1E1DA0655
:102BD000A1E0EA06F10410F461E0CFCFB0EACB1631
:102BE000B6E8DB06B1E0EB06F10410F463E0C5CF14
:102BF00065E0C3CF10ED180F1A3008F03ACFE1E0CE
:102C0000F0E0EC0FFD1F24E0029FE00DF11D112408
:102C10002081318142815381AAE0B0E00E94822C60
:102C2000610F711D811D911D608371838283938368
:102C300020CF49885A886B887C88812C912C54013C
:102C400018CF81149104A104B10489F4C301B20125
:102C50000E94670B61E070E080E090E00E948427B2
:102C60001D8A1E8A1F8A188E312C22242A948D8D4B
:102C70009E8DAF8DB8A188169906AA06BB06D0F422
:102C80000E94210B2D893E894F89588D280F311DB7
:102C9000411D511D2D8B3E8B4F8B588F381608F4DC
:102CA000382E821508F4282E3FEF831A930AA30AC0
:102CB000B30A56C0C301B20128EE33E040E050E051
:102CC0000E94B92CBA01A9012AE030E083EB95E01B
:102CD0000E94042A6CE283EB95E00E941F294AE0DF
:102CE00050E0632D83EB95E00E94132A6CE283EBA6
:102CF00095E00E941F296D897E898F89988DA50195
:102D000094010E94B92CBA01A9012AE030E083EBBA
:102D100095E00E94042A6CE283EB95E00E941F2953
:102D20004AE050E0622D83EB95E00E94132A6CE2AA
:102D300083EB95E00E945F294C0C5D1C6E1C7F1C90
:102D4000898D9A8DAB8DBC8D84159505A605B7052B
:102D500020F449885A886B887C88812C912C5401F6
:102D600029893A894B895C89283E334041055105C0
:102D700009F07FCEA296E2E10C94162DACE1B0E012
:102D8000E4ECF6E10C94042D0E9461276B017C01B8
:102D900081E00E94D70B14E703E0198361E0CE01C4
:102DA00001960E94340D0093A5050E94B20C6AEFB3
:102DB00070E080E090E00E9484278091A505833038
:102DC00089F483EB95E00E94612A892B59F40E94D3
:102DD00061276C197D098E099F096038734C894CF5
:102DE0009140D8F28091A505833009F44FC08FE758
:102DF0000E94D00A0E94E30A8983843511F083E09F
:102E00005CC00E94E30A10921805809319050E9485
:102E1000E30A2091180530911905280F311D3093D0
:102E20001905209318050E94E30A80931A050E9451
:102E3000E30A80931B05813110F7F12C0F2D10E070
:102E400080911B0590E0880F991F0817190740F41F
:102E50000E94E30AF801E45EFA4F8083F394EECF18
:102E600080E7898361E0CE0101960E94340D83E002
:102E70008093A5050E94B20C62E370E080E090E0D0
:102E80000E9484278091A505833011F482E015C04B
:102E90008FE70E94D00A0E94E30A8983803509F0F7
:102EA000AECF0FE615E00E94E30AF80181938F018F
:102EB000F5E00A381F07B9F781E06C96E8E00C945A
:102EC000202D80911705992787FD9095A92FB92F5F
:102ED000FC013196EB30F10508F066C0EC5CFF4F69
:102EE0000C94312D62E778E083EB95E00E943B295A
:102EF00084E793E00E94890D6AE578E083EB95E032
:102F00000E943B2965E378E083EB95E00E943B2932
:102F10006BE078E083EB95E00E943B296AEE77E076
:102F200083EB95E00E943B296DEB77E083EB95E026
:102F30000E943B2967E977E083EB95E00E943B29FB
:102F400063E777E083EB95E00E943B296CE477E050
:102F500083EB95E00E943B2983EB95E00E942729B3
:102F60000E94C40D21C06FE277E01AC06AE077E0EA
:102F700017C065EF76E014C066ED76E011C062E937
:102F800076E00EC06DE776E00BC068E676E083EB96
:102F900095E00E943B2962E276E002C06CE076E0B8
:102FA00083EB95E00E943B296AE070E080E090E0CE
:102FB0000E94842783EB95E00E94612A892B29F0E7
:102FC00083EB95E00E948E2AF5CF0895ACE1B0E046
:102FD000ECEEF7E10C94042D909117059F3F09F05A
:102FE00023C1482F50E0FA013A97EF36F10508F077
:102FF0000FC1E15CFF4F0C94312D63EE71E0A0C076
:103000006FEE71E083EB95E00E944D2985E789839F
:103010008BE1EFE6F5E0DE01129601900D928A95C4
:10302000E1F76CE1CE0101960E94340D0E94B20CD2
:1030300083E08093A50568EC70E080E090E00E945A
:1030400084278091A505843009F0E2C08FE70E94B3
:10305000D00A0E94E30A8983853509F0D9C06DEE54
:1030600074E083EB95E00E943B296FEC74E083EB06
:1030700095E00E943B2961EB74E096C067E072E046
:1030800083EB95E00E944D2989E6898361E0CE01BA
:1030900001960E94340D0E94B20C83E08093A50536
:1030A00068EC70E080E090E00E9484278091A505A4
:1030B000843009F0ADC08FE70E94D00A0E94E30A75
:1030C00089838E010E5F1F4F7E014DE1E40EF11CDE
:1030D0000E94E30AF80181938F01EE15FF05C1F705
:1030E0008BE1FE013296AFE6B5E001900D928A9534
:1030F000E1F78981893409F08BC063E974E083EBDF
:1031000095E00E943B2965E774E083EB95E00E941F
:103110003B2967E574E048C061E272E083EB95E02B
:103120000E944D298EEF8093170572C08052875000
:10313000805390911A05981708F066C060E372E01A
:1031400083EB95E00E944D2963C084E180931705CD
:1031500060E274E029C085E18093170569EE73E0B1
:1031600023C086E18093170562EB73E01DC087E101
:103170008093170568E673E017C088E18093170510
:1031800067E573E011C089E18093170563E473E09C
:103190000BC08AE1809317056EE273E005C08BE1F6
:1031A0008093170566E073E083EB95E00E943B296E
:1031B0002FC06CEE72E083EB95E00E943B2980917A
:1031C0007D0591E01DC066ED72E083EB95E00E9405
:1031D0003B2980917D0592E013C061EC72E083EBA6
:1031E00095E00E943B2980917D0594E009C066EA44
:1031F00072E083EB95E00E943B2980917D0598E089
:10320000892780937D058FEF809317050E946510B5
:1032100083EB95E00E94612A892B09F45BC183EB63
:1032200095E00E948E2AF4CF0E946411882309F44D
:1032300051C18091B104811104C08FEF80931705B3
:1032400041C140E050E060E070E082EB94E00E9419
:10325000A82D40911705042F112707FD1095212F48
:10326000312FF8013197EB31F10508F01BC1E25520
:10327000FF4F0C94312D552747FD509520911A058D
:1032800030E0241735070CF40DC18B019C0101506F
:10329000110921093109003211052105310558F0C4
:1032A000C0901B05EDE1F5E0F12CD12CA8E2EA2E4F
:1032B000415051090FC0FA01E159FA4F6150608342
:1032C000D9C0DF0111972C9130E02417350729F080
:1032D000F3943296FC10F5CFCBC00E2D10E020E019
:1032E00030E0061717072807390741F42081DA0173
:1032F000A159BA4F11962C93DD24D394E394E8CFCF
:103300006F3F71058105910511F008F0CBC0609306
:103310008705B0C06F3F71058105910511F008F078
:10332000C1C060938805A6C06F3F710581059105F6
:1033300011F008F0B7C0609389059CC02091B204D9
:1033400020622037E9F440E050E060E070E083EB79
:1033500094E00E94A82D9B01AC01DC01CB010197F8
:10336000A109B1090897A105B10508F0AEC0A4ED07
:10337000B0E30E94822C6A5E7C4A8A46954E24C045
:103380002636E9F440E050E060E070E083EB94E042
:103390000E94A82D9B01AC01DC01CB010197A10982
:1033A000B1090797A105B10508F08FC0A8EAB1E6F9
:1033B0000E94822C645E7C438E46944E05C061154B
:1033C00071058105910579F08B019C010054114E26
:1033D0002D4938410138F0EF1F07FAEF2F07F2E0CF
:1033E0003F0708F05FC060937F057093800580936E
:1033F0008105909382053EC06F3F7105810591055F
:1034000011F008F04FC06093830534C08B019C011C
:1034100001501109210931090F3F1105210531051D
:1034200008F040C06093840525C08B019C01045CBA
:103430001940210931090D344DE1140721053105E9
:1034400028F4709386056093850514C06115710595
:103450008105910521F48FEF80937E050BC06134C7
:10346000710581059105F0F4615060937E0502C0FD
:10347000DD20C1F08091B00481111AC080914F0508
:1034800090915005A0915105B09152050196A11D52
:10349000B11D80934F0590935005A0935105B093B3
:1034A000520506C062E472E083EB95E00E944D296C
:1034B0000E945A118FEF809317056AE083EB95E025
:1034C0000E945F290E94651005C061E070E080E005
:1034D00090E07ACF6C96E8E00C94202D6AE572E0DB
:1034E00083EB95E00E943B2962E472E083EB95E078
:1034F0000E943B2983EB95E00E94612A892B31F0E1
:1035000083EB95E00E948E2A0E94E6170E94BE1669
:10351000823029F0833051F46DE072E002C064E241
:1035200072E083EB95E00E943B2908958FEF809332
:1035300017051092B0040E946510809117058E3F08
:1035400069F083EB95E00E94612A892BB1F383EB4C
:1035500095E00E948E2A0E94E617EFCF08950F9300
:103560001F93109117051F3F09F0D1C0893409F44A
:1035700057C000F5883309F468C058F4803309F463
:1035800076C008F060C08B3109F440C08132B1F1DF
:10359000B8C0813409F486C030F4893309F465C0B9
:1035A000803461F1AEC0823409F48DC0863409F4F0
:1035B00047C0A7C0823609F486C078F4883531F157
:1035C00028F48235C1F18335E1F09BC08A3509F4D6
:1035D00093C0813609F466C094C0823761F128F443
:1035E000863671F18936E1F08CC0883779F08A37F8
:1035F00009F482C0833709F084C003C063EE71E030
:1036000015C00E94040960E672E004C00E940D0922
:103610006AE772E083EB95E00E944D298EEF6FC060
:103620000E94DC070E944B0869E972E083EB95E099
:103630000E944D2966C00E946B0862EB72E0F6CFD3
:103640000E940F115EC080535AC06AEF71E083EB95
:1036500095E00E943B2990916E0588E0890F887162
:10366000977E892B80936E051AC089E048C067EE6B
:1036700071E083EB95E00E943B2980918F0590914A
:103680009005A0919105B091920520E18227809349
:103690008F0590939005A0939105B0939205109398
:1036A00017052FC061ED71E083EB95E00E943B2987
:1036B00080918F0590919005A0919105B091920510
:1036C00040E4842710C060EC71E083EB95E00E9439
:1036D0003B2980918F0590919005A0919105B09123
:1036E000920520E2822780938F0590939005A09306
:1036F0009105B093920502C00E946E1A8FEF8093DD
:103700001705809117058E3F09F0D4C0DDC00E94D7
:103710006411882309F4D8C08091B104811104C0D8
:103720008FEF80931705C6C040E050E060E070E086
:1037300082EB94E00E94A82D00911705112707FD48
:103740001095212F312FF8013197E930F10508F05C
:10375000B4C0E753FF4F0C94312D8B019C010154F1
:10376000114E2D4938410F37104F2A4F324008F083
:10377000A4C060934B0570934C0580934D059093C6
:103780004E0577C060934F057093500580935105A7
:103790009093520581E08093B0046BC0683071054E
:1037A0008105910508F089C06093530562C08B01C3
:1037B0009C0101501109210931090A301105210527
:1037C000310508F07AC06093540553C061EB71E095
:1037D00082EB94E00E94E22E10E0009799F00E94A4
:1037E000BC2E009779F0183130F4E12FF0E0EA5B5D
:1037F000FA4F87871F5F61EB71E080E090E00E94E5
:10380000E22EEBCF1831A8F5E12FF0E0EA5BFA4F9A
:1038100017861F5FF7CF653071058105910508F0A8
:103820004CC060936D0525C08B019C0101501109AE
:10383000210931090630110521053105F0F52091E6
:103840006E05287F262B20936E0513C08B019C01EB
:1038500001501109210931090115124C214031058E
:1038600060F56093470570934805809349059093F0
:103870004A058091B004811113C080914F05909149
:103880005005A0915105B09152050196A11DB11DA1
:1038900080934F0590935005A0935105B093520526
:1038A0000E945A118FEF809317056AE083EB95E031
:1038B0000E945F290E94611707C062E472E083EBF7
:1038C00095E00E944D29ECCF1F910F9108958FEF45
:1038D000809317051092B0040E946117809117051C
:1038E0008E3F69F083EB95E00E94612A892BB1F34A
:1038F00083EB95E00E948E2A0E94AF1AEFCF6AE018
:1039000070E080E090E00E94842783EB95E00E94C5
:10391000612A892B29F083EB95E00E948E2AF5CF4E
:103920000895CF93C82F682F83EB95E00E94BB2AA0
:1039300090913C059C2790933C05CF910895A1E080
:10394000B0E0E5EAFCE10C940A2D99830E94911CF9
:103950009981892F0E94911C2196E2E00C94262DDA
:103960001F93CF93DF93182FEB0110923C0565EB6B
:1039700070E083EB95E00E94590662E670E083EB0D
:1039800095E00E945906812F0E94911CCE010E9451
:103990009F1CDF91CF911F91089560913C0583EBAF
:1039A00095E00E94BB2A0895A1E2B0E0EAEDFCE1B7
:1039B0000C94062D7B018A018B3009F42DC108F08F
:1039C0003FC0853009F49BC010F5823009F47EC0F9
:1039D00058F4813009F02FC269E270E081E00E9462
:1039E000B01C06E415E068C0833009F480C0843060
:1039F00009F021C261E070E084E00E94B01C81E027
:103A00000E94911C0E94CD1C0E94F1141EC288309D
:103A100009F49BC070F4863009F48DC0873009F03A
:103A20000AC261E070E087E00E94B01C80911A0534
:103A300008C2893009F491C08A3009F4C3C0FBC1BF
:103A4000893609F468C178F4863609F419C120F47E
:103A5000853609F401C1EFC1873609F425C18836DE
:103A600009F42AC1E8C18C3609F49EC190F48A3663
:103A700009F45BC18B3609F0DEC161E070E08BE6D2
:103A80000E94B01CF80180810E9433080E940D0939
:103A9000BDC18D3609F4BCC1873C09F0CCC161E0E1
:103AA00070E087EC0E94B01C81E00E94911C0E9493
:103AB000CD1C10923D05C9C1F80181918F010E9472
:103AC000911CF5E00F361F07B9F7BDC16BE170E03F
:103AD00082E00E94B01C0FE615E0F80181918F0191
:103AE0000E94911CF5E00A381F07B9F7ACC161E0EC
:103AF00070E083E00E94B01C0E94BE16A2C16091DB
:103B00001B0570E0660F771F85E00E94B01C0CE17A
:103B100015E080911B0590E0880F991F98012C51AA
:103B200035402817390708F08EC1F80181918F01BF
:103B30000E94911CEECF62E070E086E00E94B01C13
:103B400084E793E00E949F1C7EC161E070E088E002
:103B50000E94B01C8091A30574C186E6898361E050
:103B6000CE0101960E94340D0E94B20C83E0809336
:103B7000A50568EC70E080E090E00E9484278091C9
:103B8000A5058430D9F48FE70E94D00A0E94E30A89
:103B90008983863469F460E270E089E00E94B01C99
:103BA00010E20E94E30A0E94911C1150D1F74BC110
:103BB00061E070E089E00E94B01C28C161E070E023
:103BC00089E03CC169E170E08AE00E94B01C10927B
:103BD0008A052091A40580918F0590919005A09170
:103BE0009105B0919205222311F0806801C08F7772
:103BF00080938F0590939005A0939105B0939205C3
:103C00000AE815E0F80181918F010E94911CF5E00E
:103C1000033A1F07B9F717C161E270E08BE00E9419
:103C2000B01C80917C048F3F39F080917C0491E03E
:103C3000980F90937C0402C080917C040E94911C98
:103C400010E0812F0E94D2140E94620A0E949F1CE1
:103C50001F5F1031B1F7F7C061E070E085E60E94A8
:103C6000B01C89E2E816F10409F0EAC0D801E6E4E4
:103C7000F5E08D91819385E0EF36F807D1F7C6C066
:103C800061E070E086E60E94B01CEBE1EE16F10404
:103C900009F0D6C0D801EFE6F5E08D91819385E07B
:103CA000EA38F807D1F7B2C061E070E087E60E9419
:103CB000B01C0E940409AAC061E070E088E60E947E
:103CC000B01C85E789838BE1EFE6F5E0DE01129613
:103CD00001900D928A95E1F76CE1CE0101960E9468
:103CE000340D0E94B20C83E08093A50560E273E07E
:103CF00080E090E00E9484278091A505843009F03F
:103D00009FC08FE70E94D00A0E94E30A898385350D
:103D100009F096C07BC061E070E089E60E94B01CAB
:103D20000E94DC070E944B0871C061E070E08AE6E7
:103D30000E94B01C89E6898361E0CE0101960E9451
:103D4000340D0E94B20C83E08093A50560E273E01D
:103D500080E090E00E9484278091A505843009F0DE
:103D60006FC08FE70E94D00A0E94E30A89838E0108
:103D70000E5F1F4F7E01EDE1EE0EF11C0E94E30A83
:103D8000F80181938F01EE15FF05C1F78BE1FE016C
:103D90003296AFE6B5E001900D928A95E1F7898100
:103DA000893409F04DC032C061E070E08CE60E94B9
:103DB000B01CF0E2EF16F10461F487E6898380E23B
:103DC000F801DE01129601900D928A95E1F761E209
:103DD00003C087E4898361E0CE0101960E94340D1F
:103DE0000E94B20C83E08093A5056CE474E080E04F
:103DF00090E00E9484278091A505843009F58FE723
:103E00000E94D00A0E94E30A8734D1F481E019C0ED
:103E100061E070E08DE60E94B01C89E1E816F104D3
:103E200079F4D801EAE8F5E08D91819385E0E33AF1
:103E3000F807D1F7EBCF61E070E08AEC0E94B01C8C
:103E400080E00E94911C0E94CD1CA196E6E00C949B
:103E5000222DA0E0B0E0EFE2FFE10C94042DCCE9CC
:103E6000D3E014E606E035E0F32E44E0E42E53E020
:103E7000D52E62E0C62E83EB95E00E94612A892B45
:103E800009F49BC083EB95E00E948E2A282F809333
:103E900007044091060450E04730510560F7FA01ED
:103EA000EE52FF4F0C94312D853B29F781E0809332
:103EB0000604E1CF823609F07DC0C0920604DBCF54
:103EC0008093050480930404D0920604D4CF9C010F
:103ED000332730930304209302049091040498271D
:103EE00090930404E0920604C6CF382F2227409115
:103EF000020450910304242B352B309303042093A8
:103F0000020490910404982790930404F09206040C
:103F10002536310508F4AFCF61E070E08CEC0E94EB
:103F2000B01C81E00E94911C0E94CD1C43C02091D6
:103F3000000430910104F901E456FC4F8083909114
:103F40000404982790930404C901019690930104F6
:103F50008093000420910204309103048217930798
:103F600008F489CF0093060486CF8091040482135D
:103F70000BC060910004709101044CE953E0809102
:103F800005040E94D41C0DC062E070E08BEC0E941E
:103F9000B01C809105040E94911C80913C050E94F8
:103FA000911CFE01812F11928A95E9F7109201046C
:103FB00010920004109206045ECFCDB7DEB7E8E0A1
:103FC0000C94202D81E080933D0580913D05882350
:103FD00049F083EB95E00E94612A892BB1F30E949E
:103FE000291FF3CF0895AAE2B0E0E9EFFFE10C94B6
:103FF000022D0E9455276B017C0181E00E94D70BA6
:1040000083EB95E00E94612A892B29F083EB95E0F0
:104010000E948E2AF5CF439811E072E6B72EE9E2AE
:10402000AE2E03E00E9455276C197D098E099F0969
:10403000693C710581059105D0F11123C1F10E9400
:1040400055276B017C01429A80ED97E00E9478062B
:10405000B982E6E4F5E0DE0112968A2D01900D9218
:104060008A95E1F76AE2CE0101960E94340D4298EA
:1040700080E090E00E9478060093A5050E94B20CB3
:1040800062E370E080E090E00E9484278091A505C3
:10409000843061F40093A5058FE70E94D00A0E9446
:1040A000E30A11E0823419F410E001C011E082E16A
:1040B0000E947A28892B81F411E00EC0439A429A1B
:1040C00083EB95E00E948E2A8D309105A9F05CF477
:1040D0000A9791F04398429883EB95E00E94612AF9
:1040E000892B61F79FCF8332910579F08234910556
:1040F00089F70E94E21FEECF62EB71E083EB95E05F
:104100000E943B290E94671CE5CF0E94F114E2CF78
:104110008F929F92AF92BF92CF92DF92EF92FF92D7
:104120001F93CF93DF9382E10E947A28892B09F0B5
:1041300078C068EC70E080E090E00E94842780E026
:1041400090E00E9478060E9455274B015C016B01AC
:104150007C0180ECC80E82E1D81EE11CF11C0E949B
:1041600055276C157D058E059F0530F482E10E9470
:104170007A28892BA1F353C082E10E947A28892BE7
:1041800009F04DC080ED97E00E9478060E94552707
:104190006B017C01D0E0C1E088E4880E86E2981EC5
:1041A000A11CB11C11E082E10E947A28892B21F523
:1041B0008C149D04AE04BF0430F480ED97E00E949F
:1041C0007806D1E0F0CF0E9455276C197D098E0941
:1041D0009F09693C71058105910528F30E945527C7
:1041E0006B017C01C12719F080ED97E002C080E0EF
:1041F00090E00E947806D7CF80E090E00E94780699
:10420000DD2349F08091A3058F5F83700E943308FE
:104210000E940D0906C00E946B080E9404090E94BA
:10422000F31FDF91CF911F91FF90EF90DF90CF9020
:10423000BF90AF909F908F900895CF92DF92EF92B2
:10424000FF9280E00E94DF060E94B60661E081E1F5
:104250000E940E2861E080E10E940E2860E082E169
:104260000E940E2860E088E00E940E2861E088E04D
:104270000E9447280E94610640E052EC61E070E035
:1042800083EB95E00E94A92B0E9426080E940D094D
:104290000E94B5128FEF80937C040E94CB06789425
:1042A0000E9455276B017C0180917C048F3F59F45B
:1042B0000E9455276C197D098E099F09603D774042
:1042C0008105910588F380ED97E00E94780661E012
:1042D00082E10E944728439A83EB95E00E94612A7D
:1042E000892B29F083EB95E00E948E2AF5CF6FECA5
:1042F00072E083EB95E00E941C2984E793E00E9422
:10430000890D66EE72E083EB95E00E941C294AE07D
:1043100050E068E070E083EB95E00E94EC2962E3F6
:1043200070E080E090E00E94842783EB95E00E949B
:10433000612A04970CF183EB95E00E948E2A823467
:104340009105D1F483EB95E00E948E2A8E3491057D
:1043500099F483EB95E00E948E2A8434910561F4F0
:1043600083EB95E00E948E2A819731F480E090E003
:104370000E9478060E94F31F40914705509148051E
:104380006091490570914A05DB01CA010197A109B5
:10439000B1090497A105B10568F440937B0443304B
:1043A00029F440EA56E861E070E004C040E052ECD5
:1043B00061E070E083EB95E00E94A92B0E948820C9
:1043C000439880E090E00E9478060E94B512109217
:1043D000970480918F0583FF11C080915B0588232E
:1043E00051F080916205882331F08091690588231E
:1043F00011F087E001C085E08093970480E00E947F
:10440000D70B809198040E940B0B0E94B20C109263
:1044100011041092100410920F04F12C8091A30546
:104420008F15B0F062E370E080E090E00E94842796
:1044300080ED97E00E94780662E370E080E090E013
:104440000E94842780E090E00E947806F394E6CFF3
:1044500080916E0584FF08C0982F987181E0983193
:1044600009F080E00E94D2118FE00E94DF06FF90E9
:10447000EF90DF90CF900895EF92FF920F931F93EC
:10448000CF93DF938C016EE770E083EB95E00E94A1
:104490005906E801F12CF0E2EF2E8E0188818D574C
:1044A000823048F46DE770E083EB95E00E94590696
:1044B00088818E2588832196F801608183EB95E0C1
:1044C0000E94BB2AF394F9E0FF12E7CF6EE770E099
:1044D00083EB95E00E945906CDB7DEB7E6E00C9479
:1044E000222DA9E0B0E0E7E7F2E20C940A2D9091CA
:1044F000990491110EC09EEF99838A836B8350E0DB
:10450000559547954C832D83198618861F821E82E8
:104510002EC040919E04842F90E0B4E0959587953D
:10452000BA95E1F7242F2F7030E08217930719F125
:104530008DEF89831B82FE01349650E0842F90E03A
:10454000A4E095958795AA95E1F7242F2F7030E088
:104550008217930749F0DC01A156BB4F8C918193E0
:10456000405F5F5F563051F740939E045A83CE01FF
:1045700001960E943C228091990490E0019666E0A9
:1045800070E00E94A52C809399042996E2E00C9497
:10459000262DA0E0B0E0EFECF2E20C94032D6C01CC
:1045A0006EE770E083EB95E00E9459068601E12CEE
:1045B000F12CC0E0D0E030E2B32EF801608183E856
:1045C000860F823078F46DE770E083EB95E00E940F
:1045D0005906F80160816B2570E083EB95E00E943D
:1045E000590604C083EB95E00E94BB2AE114F10454
:1045F00059F0F80180819E01280F311DC901C92F92
:10460000DD27C80FD91FDD273FEFE31AF30A89E042
:10461000E816F10459F028E0E216F10421F48C2F99
:104620008095F60180870F5F1F4FC7CFCDB7DEB7EC
:10463000E9E00C941F2DA9E0B0E0E1E2F3E20C9474
:104640000A2DE82F362F8091990490E0019664E2BC
:1046500070E00E94A52C8093990458E9598350E199
:104660005A83813089F048F08230B9F08330D9F430
:104670008B8381EF8C833D8319C085E08B8381EF31
:104680008C832F5F2D8312C08B8381EF8C8384E614
:10469000489FA00111245D8309C084E08B8381EFD2
:1046A0008C83ED8303C00E940F1204C0CE010196DB
:1046B0000E94C9222996E2E00C94262DA2E0B0E0E7
:1046C000E4E6F3E20C94FF2C182F762E2A8349831C
:1046D0000E9461276B017C018091AF0480909A0455
:1046E00090909B04A0909C04B0909D042A814981E5
:1046F0008823C1F0D701C60188199909AA09BB0905
:104700004C015D0191EE89169EE29906A104B10467
:1047100020F1241708F4422F202F672D812F0E94AB
:104720001B2313C0D701C60188199909AA09BB091F
:104730004C015D0191E3891695E79906A104B10446
:1047400060F0672D812F0E947122C0929A04D0924E
:104750009B04E0929C04F0929D042296EDE00C9460
:104760001B2DA2E2B0E0E7EBF3E20C94002D8CE00D
:104770000E94F20A81110DC06EEE72E083EB95E0AB
:104780000E944D29439A80E00E94D70B0E94B20CF0
:10479000439883EB95E00E94612A892B01F183EB1A
:1047A00095E00E948E2A90917B04992319F00E9433
:1047B000DA12EFCF4091100450E09A012F5F3F4F83
:1047C0002F7133276091110470E02617370709F322
:1047D000FA01E55EFB4F808320931004DACF8091CD
:1047E000A505843009F086C00E9461276115710516
:1047F0008105910549F06093890470938A04809340
:104800008B0490938C040CC081E090E0A0E0B0E0B9
:104810008093890490938A04A0938B04B0938C04B2
:1048200080917F04909180048160909380048093B4
:104830007F0483E08093A5058FE70E94D00A0BE3F5
:1048400014E00E94E30AF80181938F01F4E004343C
:104850001F07B9F72091440480913B04982F9227B9
:1048600096FF3BC090E4922790934404982F98734E
:104870009833F1F410E0212F30E080913B048770F1
:1048800090E0821793074CF11F5F20916E05812FF6
:1048900090E0FC01E55CFB4F24FF04C080810E9496
:1048A000F111E9CF608183EB95E00E94BB2AE3CF51
:1048B0008F7399F480913C048093880480913D0427
:1048C0008093860480913E04809385048091410406
:1048D00090E090937E0480937D0480910F0481305A
:1048E00019F482E080930F0480910F04833011F457
:1048F00010920F040E9461276B017C01809181045A
:1049000090918204A0918304B09184040097A10542
:10491000B105C9F0A7019601281B390B4A0B5B0BA7
:10492000DA01C901883B9B40A105B10560F00E94F6
:10493000210B8093870410928104109282041092BC
:1049400083041092840480918D0490918E04A09130
:104950008F04B091900446015701881A990AAA0A57
:10496000BB0A86E495E00E944D0986169706A806C4
:10497000B90608F4A4C0C0928D04D0928E04E092CF
:104980008F04F09290040E94570680917C04883036
:10499000A0F080918F0590919005A0919105B09124
:1049A00092056CE1B695A795979587956A95D1F78D
:1049B000892B8A2B8B2B09F0A7C180917C048F5FF8
:1049C00080937C048091890490918A04A0918B0447
:1049D000B0918C040097A105B105F1F0C81AD90A6D
:1049E000EA0AFB0A86E495E00E944D096C157D05F4
:1049F0008E059F0508F002C180918F0584FD04C0DB
:104A000080ED97E00E9478061092890410928A0443
:104A100010928B0410928C0490914404907C90939B
:104A20004404509110048091110420910F045817F0
:104A300009F401C1223009F0FEC09058909344045B
:104A4000E0916E05E770F0E0E45BFC4F6081693057
:104A500008F0D9C0615040E04613D7C080931104DC
:104A600087E3840F90914404892B809344044093FE
:104A7000120483E080930F04429A9091970491115D
:104A80002DC1809198040E940B0BE0916E05E77098
:104A9000F0E0E45BFC4F608184E494E00E94ED0C64
:104AA000E0919804EF5FE0939804E83109F429C19C
:104AB000F0E0EA5BFA4F8785882309F422C10E945F
:104AC0005C0D813069F580916E05887149F18091A6
:104AD0007F0490918004880F991F909380048093A5
:104AE0007F0483E08093A5050E94B20C0E94612799
:104AF0006093810470938204809383049093840470
:104B0000672B682B692B61F481E090E0A0E0B0E0B6
:104B10008093810490938204A0938304B0938404CF
:104B200080916E0584FF1FC080917F049091800466
:104B30008E7F0E94830A182F60917D0480918804E3
:104B40000E94D012482F612F8091870449A30E94B0
:104B5000D0120091A305282F49A16091850480916E
:104B600086040E945E234298809195048130C1F0B2
:104B700018F08230B1F1D1C082E10E947A28892BED
:104B800009F0CBC081E0809395040E945527609383
:104B90009104709392048093930490939404BDC005
:104BA00082E10E947A28892B31F50E945527C09016
:104BB0009104D0909204E0909304F09094046C19C6
:104BC0007D098E099F09693E73408105910508F4AE
:104BD000A4C082E08093950480ED97E00E9478065F
:104BE0009CC082E10E947A28892B09F496C080E05B
:104BF00090E00E947806109295048FC080E090E0CB
:104C00000E94780609CF68E026CF851709F426CFE1
:104C10004F5F242F30E090E0F901EC5BFB4FDC01AB
:104C2000A55EBB4F7C917083F901EE5EFB4F7083F4
:104C300001968F7111CF2430B1F42091120483E1D9
:104C400094E0A5E4B4E0FC013E2F381B321718F4C1
:104C500031913D93F9CF87E3820F90914404892BE2
:104C60008093440406CF80919504823069F491606A
:104C700090934404439A53E9E52E55E0F52E8E01B6
:104C80000F5F1F4FB80110C0439880910F0481112E
:104C900003C081E080930F0480910F04833059F7A3
:104CA00084E080930F04E7CFF70181917F0169A32E
:104CB0007AA30E94D214F801819391938F0169A184
:104CC0007AA1F3EAEF16F5E0FF0671F780916E0521
:104CD00045E454E087700E94D209CECE80915305FE
:104CE000882309F4CECE2091960431E0320F309320
:104CF0009604291303C01092960481500E94D20B8F
:104D0000C0CE10929804DBCE80917C04883009F4E8
:104D1000439A89E080937C04D2CEA296ECE00C9476
:104D20001C2D8230E8F4E82FF0E0EE0FFF1FEA556B
:104D3000FA4F71836083813041F0809169008C7FEC
:104D4000842B80936900E89A089580916900440F4C
:104D5000551F440F551F837F842B80936900E99A68
:104D600008951F920F920FB60F9211242F933F9325
:104D70004F935F936F937F938F939F93AF93BF9363
:104D8000EF93FF938091A6059091A705892B29F0B9
:104D9000E091A605F091A7050995FF91EF91BF91CC
:104DA000AF919F918F917F916F915F914F913F91C3
:104DB0002F910F900FBE0F901F9018951F920F927A
:104DC0000FB60F9211242F933F934F935F936F93DE
:104DD0007F938F939F93AF93BF93EF93FF938091B4
:104DE000A8059091A905892B29F0E091A805F091DB
:104DF000A9050995FF91EF91BF91AF919F918F9177
:104E00007F916F915F914F913F912F910F900FBEC6
:104E10000F901F9018951F920F920FB60F921124AA
:104E20002F933F938F939F93AF93BF938091AB0545
:104E30009091AC05A091AD05B091AE053091AA0559
:104E400023E0230F2D3720F40196A11DB11D05C0CD
:104E500026E8230F0296A11DB11D2093AA05809379
:104E6000AB059093AC05A093AD05B093AE058091D2
:104E7000AF059091B005A091B105B091B205019632
:104E8000A11DB11D8093AF059093B005A093B1050E
:104E9000B093B205BF91AF919F918F913F912F91A8
:104EA0000F900FBE0F901F9018952FB7F894609138
:104EB000AB057091AC058091AD059091AE052FBF0B
:104EC00008953FB7F8948091AF059091B005A091F7
:104ED000B105B091B20526B5A89B05C02F3F19F0CA
:104EE0000196A11DB11D3FBF6627782F892F9A2FEC
:104EF000620F711D811D911D42E0660F771F881F93
:104F0000991F4A95D1F70895CF92DF92EF92FF92C1
:104F1000CF93DF936B017C010E946127EB01C114E9
:104F2000D104E104F10479F00E9461276C1B7D0B30
:104F3000683E7340A0F381E0C81AD108E108F10887
:104F4000C851DC4FECCFDF91CF91FF90EF90DF9015
:104F5000CF900895789484B5826084BD84B58160D3
:104F600084BD85B5826085BD85B5816085BDEEE671
:104F7000F0E0808181608083E1E8F0E01082808150
:104F800082608083808181608083E0E8F0E08081BE
:104F900081608083E1EBF0E0808184608083E0EBDE
:104FA000F0E0808181608083EAE7F0E080818460C6
:104FB0008083808182608083808181608083808122
:104FC000806880831092C1000895833081F028F4B6
:104FD000813099F08230A1F008958630A9F08730B1
:104FE000B9F08430D1F4809180008F7D03C080912E
:104FF00080008F7780938000089584B58F7702C0FA
:1050000084B58F7D84BD08958091B0008F7703C0F3
:105010008091B0008F7D8093B0000895CF93DF938F
:1050200090E0FC01ED50F44F2491FC01E95FF34F57
:105030008491882349F190E0880F991FFC01E15D7C
:10504000F34FA591B4918B5D934FFC01C591D49121
:105050009FB7611108C0F8948C91209582238C939E
:10506000888182230AC0623051F4F8948C91322FE7
:10507000309583238C938881822B888304C0F89495
:105080008C91822B8C939FBFDF91CF910895A1E0EB
:10509000B0E0EDE4F8E20C94082D282F30E0F9019F
:1050A000E152F44F8491F901ED50F44F1491F9015C
:1050B000E95FF34F04910023C9F0882321F069834D
:1050C0000E94E5276981E02FF0E0EE0FFF1FEB5D06
:1050D000F34FA591B4919FB7F8948C91611103C0DF
:1050E0001095812301C0812B8C939FBF2196E4E012
:1050F0000C94242DCF93DF93282F30E0F901E15257
:10510000F44F8491F901ED50F44FD491F901E95F26
:10511000F34FC491CC2391F081110E94E527EC2F2D
:10512000F0E0EE0FFF1FE55EF34FA591B4912C91D7
:105130002D2381E090E021F480E002C080E090E047
:10514000DF91CF9108958E3008F08E5087702091B6
:105150009D0190E4299F90011124822B80937C0073
:1051600080917A00806480937A0080917A0086FD35
:10517000FCCF809178002091790090E0922B0895E7
:10518000A0E0B0E0E6ECF8E20C94042D6C017A01AA
:10519000EB01E60EF71E00E010E0CE15DF0561F032
:1051A0006991D601ED91FC910190F081E02DC6014D
:1051B0000995080F191FF1CFC801CDB7DEB7E8E098
:1051C0000C94202D6115710589F0DB010D900020F4
:1051D000E9F7AD0141505109461B570BDC01ED9138
:1051E000FC910280F381E02D0995089580E090E024
:1051F0000895EF92FF920F931F93CF93DF938C014B
:10520000FB01C0E0D0E064917F018FEFE81AF80A5B
:10521000662361F0D801ED91FC910190F081E02DC1
:10522000C8010995C80FD91FF701EDCFCE01CDB741
:10523000DEB7E6E00C94222D0E94E2280895DC01FE
:10524000ED91FC910190F081E02D099508950F9367
:105250001F93CF93DF93EC016DE00E941F298C0117
:105260006AE0CE010E941F29800F911FDF91CF912C
:105270001F910F9108950F931F93CF93DF93EC012C
:105280000E94F9288C01CE010E942729800F911FCE
:10529000DF91CF911F910F9108950F931F93CF939B
:1052A000DF93EC010E94E2288C01CE010E942729A5
:1052B000800F911FDF91CF911F910F9108950F9350
:1052C0001F93CF93DF93EC010E941F298C01CE0125
:1052D0000E942729800F911FDF91CF911F910F917D
:1052E0000895A1E2B0E0E7E7F9E20C94002D7C011B
:1052F000C42EE52FCB01D22E19A221E02D1510F0DE
:105300002AE0D22E8E010F5D1F4F8D2C912CA12CE7
:10531000B12C6C2D7E2FA50194010E94B92C8C2DEF
:10532000D29E80191124015011098A3010F4805D39
:1053300001C0895CF80180832115310541055105C3
:1053400021F0C22EE32FCA01E4CFB801C7010E94A9
:10535000E228A196ECE00C941C2DA0E0B0E0E3EB79
:10536000F9E20C94042DEC016A017B012115310551
:1053700041F4E881F9810190F081E02D642F0995D5
:105380001DC02A303105A9F477FF12C06DE20E94DA
:105390001F298C0144275527BA014C195D096E0954
:1053A0007F092AE0CE010E947129800F911F06C05B
:1053B0002AE0B701A601CE010E947129CDB7DEB760
:1053C000E8E00C94202D9A01AB01662757FD60950B
:1053D000762F0E94AD2908950F931F93CF93DF93EB
:1053E000EC019A01AB01662757FD6095762F0E946C
:1053F000AD298C01CE010E942729800F911FDF91DA
:10540000CF911F910F9108952115310549F4DC01C9
:10541000ED91FC910190F081E02D642F09950895A4
:105420000E94712908959A01462F50E060E070E0D3
:105430000E94042A08959A01AB0160E070E00E9486
:10544000042A08950F931F93CF93DF93EC010E94DA
:10545000042A8C01CE010E942729800F911FDF9121
:10546000CF911F910F9108950F931F93CF93DF93C7
:10547000EC019A01AB0160E070E00E94042A8C010B
:10548000CE010E942729800F911FDF91CF911F919C
:105490000F9108950F931F93CF93DF93EC019A011F
:1054A000462F50E060E070E00E94042A8C01CE019B
:1054B0000E942729800F911FDF91CF911F910F919B
:1054C0000895FC0124853585F901E05CFF4F80815A
:1054D0009181F901EE5BFF4F20813181821B930B9B
:1054E0008F7399270895FC0184859585FC01E05C04
:1054F000FF4F40815181FC01EE5BFF4F20813181E4
:105500004217530741F00190F081E02DE80FF91F99
:10551000808190E008958FEF9FEF0895FC018485CE
:105520009585FC01E05CFF4F40815181FC01EE5B01
:10553000FF4F208131814217530779F0A081B1815B
:10554000A80FB91F8C91208131812F5F3F4F2F739E
:1055500033273183208390E008958FEF9FEF0895E4
:10556000FC0181A1882329F0A489B5898C9186FF4B
:10557000FBCF11A20895CF93DF93FC0126853785D9
:10558000D901A05CBF4F8D919C91119701968F73AB
:105590009927E901CE5BDF4F488159818417950730
:1055A000D9F30D90BC91A02DA20FB31F6C93A685CB
:1055B000B785A05CBF4F11969C938E93A689B7893F
:1055C0002C9181E090E0078C02C0880F991F0A940B
:1055D000E2F7282B2C9381E081A30488F589E02D44
:1055E00080818064808381E090E0DF91CF91089595
:1055F00008951F920F920FB60F9211242F933F938D
:105600004F938F939F93EF93FF938091C00082FD00
:105610001CC04091C6008091590690915A0601968F
:105620008F73992720915B0630915C068217930750
:1056300071F0E0915906F0915A06E75EF94F408308
:1056400090935A068093590602C08091C600FF913C
:10565000EF919F918F914F913F912F910F900FBE9E
:105660000F901F90189583EB95E00E94612A892B7B
:1056700011F00E94F82A08951F920F920FB60F9210
:1056800011242F933F938F939F93EF93FF93209138
:105690001506309116068091170690911806281766
:1056A000390731F48091C1008F7D8093C10014C00F
:1056B000E0911706F0911806EB52FA4F2081809185
:1056C00017069091180601968F73992790931806E4
:1056D000809317062093C600FF91EF919F918F91C1
:1056E0003F912F910F900FBE0F901F901895A0E043
:1056F000B0E0EDE7FBE20C94002DFC011382128276
:1057000088EE93E0A0E0B0E084839583A683B7831E
:105710008EE893E0918380837587648757874687F7
:10572000318B208B138B028BF58AE48AD78AC68A49
:10573000B18EA08E938E828E8F85848F8889858F7F
:105740008989868F8A89878F8B8980A3ECE00C9466
:105750001C2DCF92DF92EF92FF92CF93DF93EC015B
:105760006A017B01411581EE580761057105F9F069
:10577000EC89FD8981E090E008A002C0880F991FA4
:105780000A94E2F7808360E079E08DE390E0A7017E
:1057900096010E94B92C21503109410951095695B1
:1057A000479537952795211580E1380798F0EC89C2
:1057B000FD89108260E874E88EE190E0A70196010F
:1057C0000E94B92C2150310941095109569547953C
:1057D00037952795E889F9893083EA89FB89208301
:1057E00019A2EE89FF89408181E090E09C010C8C38
:1057F00002C0220F331F0A94E2F7422B4083EE8946
:10580000FF8940819C010D8C02C0220F331F0A9436
:10581000E2F7422B4083EE89FF8940819C010E8C88
:1058200002C0220F331F0A94E2F7422B4083EE8915
:10583000FF8920810F8C02C0880F991F0A94E2F71C
:10584000809582238083DF91CF91FF90EF90DF904E
:10585000CF9008958F929F92AF92BF92CF92DF9296
:10586000EF92FF920F931F9381E08F9385E08F93C8
:1058700087E08F9383E08F9384E08F93E6EC8E2E06
:10588000912CF2ECAF2EB12CA1ECCA2ED12CB0ECA5
:10589000EB2EF12C04EC10E025EC30E045ED55E06A
:1058A00069E176E083EB95E00E94772B0F900F90F3
:1058B0000F900F900F901F910F91FF90EF90DF903E
:1058C000CF90BF90AF909F908F9008950E94AA278D
:1058D0000E941D21C3E3DBE20E94B1232097E1F384
:1058E0000E94332BF9CFA29FB001B39FC001A39FA9
:1058F000700D811D1124911DB29F700D811D112409
:10590000911D08950E94732CA59F900DB49F900D3A
:10591000A49F800D911D11240895B7FF0C94822C33
:105920000E94822C821B930B0895DB018F939F931F
:105930000E94822CBF91AF91A29F800D911DA39FC9
:10594000900DB29F900D1124089597FB072E16F429
:10595000009407D077FD09D00E94372D07FC05D0B1
:105960003EF4909581959F4F0895709561957F4F76
:105970000895A1E21A2EAA1BBB1BFD010DC0AA1F90
:10598000BB1FEE1FFF1FA217B307E407F50720F0A8
:10599000A21BB30BE40BF50B661F771F881F991F23
:1059A0001A9469F760957095809590959B01AC016C
:1059B000BD01CF010895052E97FB1EF400940E94AF
:1059C000F22C57FD07D00E94B92C07FC03D04EF4EF
:1059D0000C94F22C50954095309521953F4F4F4FA8
:1059E0005F4F089590958095709561957F4F8F4F8B
:1059F0009F4F08952F923F924F925F926F927F92A6
:105A00008F929F92AF92BF92CF92DF92EF92FF92CE
:105A10000F931F93CF93DF93CDB7DEB7CA1BDB0B7A
:105A20000FB6F894DEBF0FBECDBF09942A8839881F
:105A300048885F846E847D848C849B84AA84B98426
:105A4000C884DF80EE80FD800C811B81AA81B98132
:105A5000CE0FD11D0FB6F894DEBF0FBECDBFED0146
:105A60000895EE0FFF1F0590F491E02D0994AA1BF5
:105A7000BB1B51E107C0AA1FBB1FA617B70710F039
:105A8000A61BB70B881F991F5A95A9F7809590956B
:105A9000BC01CD0108958F929F92AF92BF92CF9299
:105AA000DF92EF92FF92CF93DF93EC0168817981CF
:105AB0008A819B81611571058105910521F464E25C
:105AC00079ED8BE597E02DE133EF41E050E00E9466
:105AD000DB2C49015A019B01AC01A7EAB1E40E9409
:105AE000822C6B017C01ACEEB4EFA50194010E9405
:105AF000902CC60ED71EE81EF91EF7FE06C081E0E8
:105B0000C81AD108E10880E8F80AC882D982EA8276
:105B1000FB82C701B6019F77DF91CF91FF90EF9095
:105B2000DF90CF90BF90AF909F908F9008950E948C
:105B30004B2D089586E091E00E944B2D08956093CF
:105B4000060170930701809308019093090108955D
:105B50002F923F925F926F927F928F929F92AF921D
:105B6000BF92CF92DF92EF92FF920F931F93CF934A
:105B7000DF938B01EA016115710521F0DB018C9344
:105B800011969C93209739F09E01225031092332BF
:105B9000310508F0D8C07C016701BFEFCB1ADB0AE2
:105BA0005601F7016080862D90E00E94DA2E892B45
:105BB00011F07601F1CFFDE26F120AC0570182E0C9
:105BC000A80EB11CD70111966C90772473940BC06A
:105BD000BBE26B1207C05701E2E0AE0EB11CD70169
:105BE00011966C90712CCE018F7E892B89F4B0E3D5
:105BF0006B1237C0F50180818F7D8835D1F46180CB
:105C0000F2E0AF0EB11C872D8260782EC0E1D0E0AB
:105C1000CA30D10551F1C031D10521F0C830D105CC
:105C200099F409C0CC24CA94DC2CEC2CAFE0FA2EF9
:105C300022C0209769F7C8E0D0E0CC24CA94DC2CBD
:105C4000EC2CFFE1FF2E17C06FEF7FEFCB019E0121
:105C5000442737FD4095542F0E94B92C69017A01E1
:105C60000AC02097A9F6CAE0D0E0E9E9CE2EDC2CE4
:105C7000EC2CE9E1FE2EF50160E020E030E0A90126
:105C80004E01AA2497FCA094BA2C1F0170ED572E48
:105C9000560CA9E0A51570F48FEB860D8A3118F427
:105CA00099EC592E06C08FE9860D8A3148F589EAAC
:105CB000582E560C852D90E08C179D070CF56F3FE4
:105CC000D9F0C216D306E406F50698F0C501B40172
:105CD0000E94952C9B01AC01852D90E0A0E0B0E0E6
:105CE000280F391F4A1F5B1F281739074A075B0710
:105CF00010F46FEF01C061E03196D1016C90C5CF17
:105D00000115110551F0662311F0319703C071FEA2
:105D100004C03297D801ED93FC9370FE07C05095F4
:105D20004095309521953F4F4F4F5F4F67FF10C013
:105D300082E290E090935E0680935D066FEF7FEFC6
:105D40008FEF9FEF07C060E070E080E090E002C05E
:105D5000B901CA01DF91CF911F910F91FF90EF9090
:105D6000DF90CF90BF90AF909F908F907F906F907B
:105D70005F903F902F900895FC0188279927E89421
:105D800021912032E9F3293010F02E30C8F32B3264
:105D900041F02D3239F4689404C00E940E2F820F16
:105DA000911D219120532A30C0F31EF490958195C6
:105DB0009F4F0895911150C0803219F0895085503D
:105DC000D0F708954AE953E00E94E72E0895FA01BA
:105DD000A191B081009719F41097E1F0CD01DC0199
:105DE000CD010D90002011F4C00113C0FB012191E1
:105DF000222319F02015D9F7F3CFFB0121912015AB
:105E000019F41E92119606C02223C1F70D900020AE
:105E1000A1F7D001FA01A193B08308957AE0979F8A
:105E2000902D879F802D910D11240895F999FECF13
:105E300092BD81BDF89A992780B50895262FF999CA
:105E4000FECF1FBA92BD81BD20BD0FB6F894FA9A5D
:105E5000F99A0FBE01960895992788270895F89416
:025E6000FFCF72
:105E620000005F06200001000000FF0002000200A7
:105E72000200020002000200020002000200020010
:105E8200020002000200020002000280250000055A
:105E9200400AA1204EA50020244EA52C2330C0127A
:105EA20000001A400AA1204EA5001B1E27522C23D7
:105EB200308025000005400AA1204EA50020244E76
:105EC200A52C2330004B000006400AD0009D49005B
:105ED2007B289D492C233000E1000005400A450142
:105EE200D7DC03B81E0EBF00232E48E801008A400B
:105EF2000A6001555502AD1E20000023C801545806
:105F02002074696D656F75742100596573004E6F59
:105F1200002C00386368004E2F41002C205B005D8E
:105F22002028002900486F70206368616E6E656CDE
:105F32002000204020007363616E6E6572206D6FD9
:105F42006465004E4F5420454E41424C4544005337
:105F5200656E64696E672073657474696E67732019
:105F6200746F2052580A00526573657474696E67C3
:105F72002073657474696E6773206F6E2052580ABD
:105F82000041626F727465642065646974730A000B
:105F9200696E76616C69642073656C656374696FA0
:105FA2006E000D0A496E76616C696420696E7075C7
:105FB20074202D2064697363617264656421070033
:105FC20053657474696E67732073617665642074B7
:105FD2006F20454550524F4D0A00526576657274E6
:105FE20065642073657474696E67732066726F6D81
:105FF20020454550524F4D0A004C6F616465642044
:10600200666163746F72792064656661756C74731E
:106012000A004B657920616E64206368616E6E656B
:106022006C732072616E646F6D697A65640A004FE9
:1060320070656E4C52536E672054582073746172AF
:1060420074696E672000206F6E20485720006D6FC4
:1060520064756C65206C6F636B65643F00342B3430
:10606200003800382B340031320031322B34003109
:10607200360050504D00525353490053444100538F
:10608200434C00525844005458440041494E004C7D
:10609200424545500053504B54524D0053425553C4
:1060A2000053554D44004C4C494E440000070B0C24
:1060B20010111500B701FD020103030307030A03D0
:1060C2000F03B701160A13223129120316031B0309
:1060D2001F03230327032B032F0335033C03410331
:1060E20046035F025F025F025F0200000000BB2AFC
:0A60F200C028612A8E2A732AB02A02
:107E00000F92CDB7DEB7112484B714BE81FFF1D035
:107E100082E08093C00088E18093C10086E0809377
:107E2000C20080E18093C4008EE0CDD088249924E4
:107E3000CC24C394F5E0DF2EE1E1EE2E73E0F72EC3
:107E4000B6D0082F813479F4B2D08983C2D0898129
:107E5000823811F481E005C0813811F485E001C059
:107E600083E09ED09AC0823411F484E103C085344B
:107E700019F485E0B6D091C0853561F498D0082F0B
:107E800010E095D090E0982E8824802A912A880CC2
:107E9000991C82C0863521F484E0A3D080E0E1CF34
:107EA000843609F04CC083D082D0A82E80D0B82E62
:107EB00000E011E07CD0F80181938F01AE16D1F77C
:107EC00088D0FB2DF53489F4E0E0F1E00BC0F9999E
:107ED000FECF92BC81BC0894811C911C819180BD15
:107EE000FA9AF99AEA1598F358C08B2D863409F05E
:107EF00054C0F401F7BEE89507B600FCFDCFF401CD
:107F0000A0E0B1E02C9130E011968C91119790E0B7
:107F1000982F8827822B932B12960C01C7BEE895C9
:107F20001124329681E0A038B80761F7F401D7BE7A
:107F3000E89507B600FCFDCFE7BEE8952EC0843774
:107F4000F1F435D034D0182F32D0B82E42D0FB2DDA
:107F5000F63421F4F40105914F010CC0FB2DF534EA
:107F600049F4F999FECF92BC81BC0894811C911C04
:107F7000F89A00B5802F14D0115049F70EC08537FC
:107F800039F427D08EE10CD085E90AD08FE069CF93
:107F9000813511F488E017D01CD080E101D050CF9A
:107FA0009091C00095FFFCCF8093C600089580910A
:107FB000C00087FFFCCF8091C00084FD01C0A89560
:107FC0008091C6000895E0E6F0E098E19083808318
:107FD0000895EDDF803219F088E0F5DFFFCF84E10E
:107FE000DFCF1F93182FE3DF1150E9F7F2DF1F9166
:0E7FF0000895282E80E0E7DFEE27FF27099492
:027FFE0001057B
:0400000300007E007B
:00000001FF
